:020000040000FA
:100000007AEF0DF0F76A140FF66E000EF722090072
:10001000F5501200280C0106F76A280FF66E000E44
:10002000F7220900F550120025346C75204C495414
:1000300052455325336C75252500F76A4A0FF66E35
:10004000000EF7220900F55012000C00F76A5C0F51
:10005000F66E000EF7220900F55012005341564586
:1000600057415445520A4649524D57415245205630
:10007000657220312E300000F76A880FF66E000E90
:10008000F7220900F550120020452E4B4F454E49EE
:1000900047554552286329200A616C706169722EA8
:1000A000667265652E667200F76AB80FF66E000E0E
:1000B000F7220900F5501200205245474C414745B0
:1000C00020484555524520200000F76ADA0FF66EA9
:1000D000000EF7220900F5501200484555524553CD
:1000E000203A202530327500F76AF80FF66E000EC0
:1000F000F7220900F55012004D494E555445532042
:100100003A20253032750000F76A180FF66E010E9E
:10011000F7220900F5501200454E52454749535405
:1001200052450000F76A340FF66E010EF7220900FF
:10013000F5501200205245474C4147452044415458
:100140004500F76A520FF66E010EF7220900F550CE
:1001500012004A4F5552203A202530327500F76A76
:100160006E0FF66E010EF7220900F55012004D4F8A
:100170004953203A202530327500F76A8A0FF66E0F
:10018000010EF7220900F5501200414E4E45452060
:100190003A203230253032750000F76AAA0FF66E29
:1001A000010EF7220900F55012004D454E550A5236
:1001B00045474C4147452048455552450000F76AA0
:1001C000CE0FF66E010EF7220900F55012004D45D4
:1001D0004E550A5245474C4147452044415445003D
:1001E000F76AF00FF66E010EF7220900F5501200C3
:1001F0004D454E550A434F4E54454E414E434520C2
:10020000435556452000F76A160FF66E020EF72288
:100210000900F5501200434F4E54454E414E4345A0
:100220002043555645200000F76A380FF66E020E3F
:10023000F7220900F55012004D454E550A4E495619
:1002400045415520454155204D494E492E00F76AFC
:100250005E0FF66E020EF7220900F55012004E49AD
:100260005645415520454155204D494E492E0000E7
:10027000F76A800FF66E020EF7220900F5501200A1
:100280004D454E550A44454C5441204E4956454132
:10029000552045415500F76AA60FF66E020EF7226B
:1002A0000900F550120044454C5441204E49564532
:1002B0004155204541550000F76AC80FF66E020E01
:1002C000F7220900F55012004D454E550A5354418E
:1002D00054495354495155455300F76AEA0FF66E95
:1002E000020EF7220900F550120025346C75204CDF
:1002F000495452455300EA6A310EE96EEF500DE061
:10030000060E016E006A002EFED7012EFBD77B0E73
:10031000006E002EFED7EF2EF3D7000C38B002D0BF
:100320008C9C01D08C8C959C38B202D08C9E01D0D4
:100330008C8E959E38B402D08A9001D08A8093909A
:1003400038B602D08A9201D08A8293920000959AA0
:100350008C8A030E006E002EFED7959A8C9A000CA4
:1003600095988C98630E006E002EFED7000000005A
:10037000355203E095988C8802D095988C980000AF
:10038000959A8C9A3638376E0F0E371637C038F07C
:10039000C5DF36500F0B376E37C038F0BFDF000CAB
:1003A00095988C98959A8C9A0F0E316EA4DF1D6AE1
:1003B0001D50020808E3030E386EB0DF050E316EE3
:1003C0009ADF1D2AF5D7020E386EA8DF1D6A1D5070
:1003D00003080DE3036A1D5015DE1E6E356A1EC04C
:1003E00036F0BEDF050E316E86DF1D2AF0D77FEFB7
:1003F00003F0322C01D003D0400E336E01D0336AAB
:10040000010E315C332633508009346E356A34C0B6
:1004100036F0A6DF000C30500C0A05E0060A0BE0AF
:10042000020A0FE013D0356A010E366E99DF020E14
:10043000316E61DF11D0010E316E020E326ED9DFE6
:100440000BD0356A100E366E8BDF06D0010E356E7E
:1004500030C036F085DF00D0000C080E016E0000C1
:10046000040E006E002EFED78B969496060E006E3C
:10047000002EFED735368B98D8B09488D8A09498A3
:10048000948682A6FED7012EEAD7040E006E002EB7
:10049000FED78B96949600009488060E006E002E70
:1004A000FED7060E006E002EFED7948682A6FED7DB
:1004B000016A060E006E002EFED782B801808B9670
:1004C00094968B989498000C080E346E00C035F00A
:1004D0009488060E006E002EFED7948682A6FED764
:1004E00082B8D88082A8D8900136040E006E002E03
:1004F000FED794968B96342EEBD79488060E006E1A
:10050000002EFED78B983550D8A49498000094867E
:1005100082A6FED7040E006E002EFED78B96949610
:10052000060E006E002EFED78B989498000C24C007
:1005300025F0D8902532780E25162530006E003231
:100540003F0E001600502524266E24500F0B262443
:10055000016E000C25C026F0276A2650090805E226
:100560000A0E265E100E272603D02650272601D01D
:10057000F4D727C001F0000C1D6A9488040E006EA9
:10058000002EFED79486060E006E002EFED78B98A6
:100590009498040E006E002EFED78B969496D00E83
:1005A000356E5BDF356A59DF9488040E006E002ECD
:1005B000FED79486060E006E002EFED78B98949878
:1005C000040E006E002EFED78B969496D10E356EDB
:1005D00044DF006A79DF01C01EF001C024F0A7DF0C
:1005E00001C01DF094980000948682A6FED7040EE8
:1005F000006E002EFED70000000000009488040E5C
:10060000006E002EFED71D9E040E006E002EFED73B
:10061000000000009488040E006E002EFED7948621
:10062000060E006E002EFED78B989498040E006E76
:10063000002EFED78B969496D00E356E0EDF356A5F
:100640000CDF1DC025F086DF01C01EF001C035F0B3
:1006500004DF9488040E006E002EFED79486060EEA
:10066000006E002EFED78B989498040E006E002E1C
:10067000FED78B969496D00E356EEFDE070E356E54
:10068000ECDE800E356EE9DE94980000948682A63A
:10069000FED7040E006E002EFED700000000000002
:1006A0009488040E006E002EFED7D9EF03F09486D6
:1006B0009488DAEF03F0C190C182C184C186C19CE5
:1006C000C28CC28EC18EC2809698D190800ED56E9B
:1006D000CD6A000E016ECA6E000ECB6EB150480B93
:1006E000B16E94928B82020E1D6E960E316E03DEF9
:1006F0001D2EFBD794928B9295928C8251D61D6AB7
:100700001D509BDC000904E01D2A306E84DEF8D702
:10071000030E1D6E2A0E306E7EDE1D2EFBD71E6A66
:100720001E5094DC1E2A006E00C030F074DE090EEC
:100730001E5CF6E1030E1F6E2A0E306E6CDE1F2E5D
:10074000FBD7090E206E205081DC202A006E00C0ED
:1007500030F061DE1A0E205CF6E1080E1D6EFA0E16
:10076000316EC9DD1D2EFBD71D6A1D5066DC0009E8
:1007700004E01D2A306E4FDEF8D71D6A1D507CDC68
:100780001D2A006E00C030F046DE1F0E1D5CF6E133
:10079000080E1D6EFA0E316EAEDD1D2EFBD71D6AE2
:1007A0001D504BDC000904E01D2A306E34DEF8D702
:1007B000E3D67DD795928C921C901C8293EF0DF01E
:1007C0002250016A215C03E221C000F00CD0006AD3
:1007D000080E236E213600362250005CD8B0006E21
:1007E0000136232EF7D7000C01501FC021F0640EF4
:1007F000226EE6DF00C01FF00150300E07E120B08E
:100800000BD020B609D020B8200E02D02096209818
:10081000012601C030F0FFDD1FC021F00A0E226E5C
:10082000CFDF00C01FF00150300E04E120B606D02B
:1008300020B8200E012601C030F0EDDD300E1F265D
:100840001FC030F0E8DD000C249E3F0E2216948875
:10085000040E006E002EFED79486060E006E002E4B
:10086000FED78B989498040E006E002EFED78B96C0
:100870009496D00E356EF1DD356AEFDD24C025F09B
:1008800069DE01C025F001C035F0E7DD23C025F0A9
:1008900061DE01C025F001C035F0DFDD22C025F0AA
:1008A00059DE01C025F001C035F0D7DD21C025F0AB
:1008B00051DE01C025F001C035F0CFDD1EC025F0AE
:1008C00049DE01C025F001C035F0C7DD1FC025F0AD
:1008D00041DE01C025F001C035F0BFDD20C025F0AC
:1008E00039DE01C025F001C035F0B7DD800E356E70
:1008F000B4DD94980000948682A6FED7040E006EA4
:10090000002EFED70000000000009488040E006E48
:10091000002EFED7000C9488040E006E002EFED729
:100920009486060E006E002EFED78B989498040EC7
:10093000006E002EFED78B969496D00E356E8DDD10
:10094000356A8BDD9488040E006E002EFED79486E7
:10095000060E006E002EFED78B989498040E006E43
:10096000002EFED78B969496D10E356E76DD010E55
:10097000006EAADD01507F0B1F6E1FC024F0D7DD73
:1009800001C005F0010E006E9FDD01507F0B1F6E50
:100990001FC024F0CCDD01C006F0006A95DD0150D7
:1009A0003F0B1F6E1FC024F0C2DD01C007F09498FA
:1009B0000000948682A6FED7040E006E002EFED79D
:1009C0000000000000009488040E006E002EFED788
:1009D000056A1E6A1E501DEC00F0000904E01E2A84
:1009E000306E19DDF7D7010E316E326E02DD1E6AF0
:1009F0001E5054EC00F01E2A006E00C030F00BDDDB
:100A0000100E1E5CF5E1C80E316E75DC9284000E8E
:100A100080B4010E000A34E0010E316E020E326E17
:100A2000E8DC1E6A1E5065EC00F01E2A006E00C055
:100A300030F0F1DC090E1E5CF5E107C01FF0010E7D
:100A4000206ED2DEFA0E316E56DC9286000E80B633
:100A5000010E000A07E10750170802E1076A02D0F9
:100A6000010E07269288000E80B8010E000A07E1E9
:100A7000075203E1170E076E02D0010E075EC6D7BC
:100A8000FA0E316E38DC9284000E80B4010E000A3A
:100A900034E0010E316E020E326EABDC1E6A1E5067
:100AA00074EC00F01E2A006E00C030F0B4DC0A0EB8
:100AB0001E5CF5E106C01FF0010E206E95DEFA0EF9
:100AC000316E19DC9286000E80B6010E000A07E135
:100AD00006503B0802E1066A02D0010E0626928803
:100AE000000E80B8010E000A07E1065203E13B0E3A
:100AF000066E02D0010E065EC6D708C01EF009C001
:100B00001FF00AC020F00BC021F007C022F006C081
:100B100023F005C024F098DE010E316E020E326E15
:100B200068DC030E1E6E200E306E75DC1E2EFBD7A9
:100B30001F6A1F5084EC00F01F2A006E00C030F0C6
:100B40006ADC0A0E1F5CF5E1030E206E200E306E8B
:100B500062DC202EFBD7080E1E6EFA0E316E7BEC87
:100B600001F01E2EFAD7AAEF09F09488040E006E49
:100B7000002EFED79486060E006E002EFED78B98B0
:100B80009498040E006E002EFED78B969496D00E8D
:100B9000356E63DC030E356E60DC9488040E006EE7
:100BA000002EFED79486060E006E002EFED78B9880
:100BB0009498040E006E002EFED78B969496D10E5C
:100BC000356E4BDC010E006E7FDC01507F0B1F6E1B
:100BD0001FC024F0ACDC01C00BF0010E006E74DC11
:100BE00001503F0B1F6E1FC024F0A1DC01C008F0B4
:100BF000010E006E69DC01501F0B1F6E1FC024F038
:100C000096DC01C009F0006A5FDC01C01EF001C083
:100C100024F08DDC01C00AF094980000948682A62E
:100C2000FED7040E006E002EFED70000000000006C
:100C30009488040E006E002EFED71E6A1E501DEC16
:100C400000F0000905E01E2A306E0BEC02F0F6D72A
:100C5000010E316E326EF9EC01F01E6A1E5092ECFC
:100C600000F01E2A006E00C030F00BEC02F00D0EFA
:100C70001E5CF4E1030E1F6E200E306E0BEC02F0D2
:100C80001F2EFAD7C80E316E7BEC01F09284000E55
:100C900080B4010E000A38E0010E316E020E326E91
:100CA000F9EC01F01E6A1E50A1EC00F01E2A006E45
:100CB00000C030F00BEC02F0070E1E5CF4E108C03F
:100CC0001FF0010E206E90DDFA0E316E7BEC01F00C
:100CD0009286000E80B6010E000A08E108501F0837
:100CE00003E1010E086E02D0010E08269288000E64
:100CF00080B8010E000A07E1082C03D01F0E086E11
:100D000002D0010E085EC2D7FA0E316E7BEC01F004
:100D10009284000E80B4010E000A38E0010E316E9C
:100D2000020E326EF9EC01F01E6A1E50AFEC00F0BC
:100D30001E2A006E00C030F00BEC02F0070E1E5CA5
:100D4000F4E109C01FF0010E206E4EDDFA0E316E87
:100D50007BEC01F09286000E80B6010E000A08E1DD
:100D600009500C0803E1010E096E02D0010E09269C
:100D70009288000E80B8010E000A07E1092C03D00A
:100D80000C0E096E02D0010E095EC2D7FA0E316E4A
:100D90007BEC01F09284000E80B4010E000A37E073
:100DA000010E316E020E326EF9EC01F01E6A1E5019
:100DB000BDEC00F01E2A006E00C030F00BEC02F01B
:100DC0000A0E1E5CF4E10AC01FF0010E206E0CDD5D
:100DD000FA0E316E7BEC01F09286000E80B6010EA9
:100DE000000A07E10A50630802E10A6A02D0010E14
:100DF0000A269288000E80B8010E000A07E10A5206
:100E000003E1630E0A6E02D0010E0A5EC3D708C06A
:100E10001EF009C01FF00AC020F00BC021F007C06F
:100E200022F006C023F005C024F00EDD010E316E65
:100E3000020E326EF9EC01F0030E1E6E200E306EC3
:100E40000BEC02F01E2EFAD71F6A1F5084EC00F044
:100E50001F2A006E00C030F00BEC02F00A0E1F5C7F
:100E6000F4E1030E206E200E306E0BEC02F0202E0B
:100E7000FAD7080E1E6EFA0E316E7BEC01F01E2EB4
:100E8000FAD7E8EF09F09488040E006E002EFED722
:100E90009486060E006E002EFED78B989498040E52
:100EA000006E002EFED78B969496A00E356E2DEC1C
:100EB00002F031C033F0346A31C035F02DEC02F06D
:100EC00030C035F02DEC02F09488040E006E002E38
:100ED000FED79486060E006E002EFED78B9894984F
:100EE000040E006E002EFED78B969496A10E356EE2
:100EF0002DEC02F0006A64EC02F001C032F094982C
:100F00000000948682A6FED7040E006E002EFED747
:100F10000000000000009488040E006E002EFED732
:100F200032C001F0000C2DC031F02CC030F0ABDF2E
:100F30002F6A01C02EF02C2AD8B42D2A2EC02FF0F3
:100F40002E6A2DC031F02CC030F09DDF01502E12E2
:100F50002EC001F02FC002F0000CEACF2FF0E9CF35
:100F60002EF02838F0092A6E2A26E20F2B6E320F57
:100F70002D6E28500F0B2B262B262D26E90F2C6EBD
:100F80002C262C2627380F0B2C262D262C362D36DA
:100F90002D1E2D3627500F0B2D262A36070E296EB3
:100FA0000A0E2C062D26FDE32B062C26FDE32A0631
:100FB0002B26FDE329062A26FDE3EA6A290EE96EBF
:100FC000070E2E14E9262D0EE95C1FE0EF50006E8F
:100FD00006E12EB818D02EB604D0200E03D0080E8D
:100FE0002E6E300E0026EACF28F0E9CF27F0005011
:100FF000296E00C030F00BEC02F028C0EAFF27C0D9
:10100000E9FF2950006EEE50DED7EF50006E300E33
:10101000002600C030F00BEC02F0000C1FC025F0E1
:101020001EC024F02680FA0E316E7BEC01F0928413
:10103000000E80B4010E000A52E0010E316E020E65
:10104000326EF9EC01F0010EE96E25C028F024C0E3
:1010500027F083DF040E276E27506DEC01F0272A5E
:10106000006E00C030F00BEC02F00B0E275CF4E1D8
:10107000050E286E200E306E0BEC02F0282EFAD7EB
:10108000960E316E7BEC01F0928680B617D022501E
:10109000245C06E12350255C03E1256A246A0ED016
:1010A000000E26B0010E010805E11E0E2426000EDA
:1010B000252204D0010E2426000E2522928880B815
:1010C0000DD0245207E1255205E123C025F022C0AE
:1010D00024F004D0010E245E000E255AA8D7010E7C
:1010E000316E020E326EF9EC01F0030E276E200E07
:1010F000306E0BEC02F0272EFAD7286A285084ECC9
:1011000000F0282A006E00C030F00BEC02F00A0E4E
:10111000285CF4E1030E296E200E306E0BEC02F019
:10112000292EFAD7080E276EFA0E316E7BEC01F0ED
:10113000272EFAD724C001F025C002F0000C9488B5
:10114000040E006E002EFED79486060E006E002E52
:10115000FED78B989498040E006E002EFED78B96C7
:101160009496A00E356E2DEC02F025C028F0296A69
:1011700025C035F02DEC02F024C035F02DEC02F046
:1011800026C035F02DEC02F094980000948682A6DB
:10119000FED7040E006E002EFED7000000000000F7
:1011A0009488040E006E002EFED79488040E006E04
:1011B000002EFED79486060E006E002EFED78B986A
:1011C0009498040E006E002EFED78B969496A00E77
:1011D000356E2DEC02F0015001B002D0279001D005
:1011E0002780000E27B0010E01081DE19488040E2F
:1011F000006E002EFED79486060E006E002EFED7DF
:101200008B989498040E006E002EFED78B969496C1
:10121000A00E356E2DEC02F0015001B002D02790E7
:1012200001D02780DED7000C21C022F0236A1FC026
:1012300025F01EC024F021C026F081DF1E2AD8B47C
:101240001F2A1FC025F01EC024F020C026F077DF23
:10125000000C1E6A1E501DEC00F0000905E01E2A5D
:10126000306E0BEC02F0F6D79286000E80B6010EBF
:10127000000A03E1010E1D6E02D0060E1D6EFA0E6D
:10128000316E7BEC01F09282000E80B2010E000AFA
:10129000D8B451D29286000E80B6010E000A08E141
:1012A0001D50060803E1010E1D6E02D0010E1D2621
:1012B0009288000E80B8010E000A07E11D2C03D0B1
:1012C000060E1D6E02D0010E1D5E010E1D5CFA0F92
:1012D000D8B02CD2060FA8EF0BF0010E316E326E93
:1012E000F9EC01F0060E1E6E2D0E306E0BEC02F0C6
:1012F0001E2EFAD71F6A1F50CDEC00F01F2A006E79
:1013000000C030F00BEC02F0040E1F5CF4E1060E9E
:10131000206E2D0E306E0BEC02F0202EFAD7040E4C
:10132000216E2150CDEC00F0212A006E00C030F07B
:101330000BEC02F0120E215CF4E1030E226E200E83
:10134000306E0BEC02F0222EFAD7928480B402D0D9
:101350008BEF04F0EBD1010E316E326EF9EC01F03F
:10136000060E1E6E2D0E306E0BEC02F01E2EFAD7FE
:101370001F6A1F50DFEC00F01F2A006E00C030F023
:101380000BEC02F0040E1F5CF4E1060E206E2D0E35
:10139000306E0BEC02F0202EFAD7040E216E215095
:1013A000DFEC00F0212A006E00C030F00BEC02F000
:1013B000110E215CF4E1040E226E200E306E0BEC57
:1013C00002F0222EFAD7928480B402D0B5EF05F055
:1013D000ADD1010E316E326EF9EC01F0060E1E6ECB
:1013E0002D0E306E0BEC02F01E2EFAD71F6A1F5026
:1013F000F0EC00F01F2A006E00C030F00BEC02F0A1
:10140000040E1F5CF4E1060E206E2D0E306E0BEC08
:1014100002F0202EFAD7040E216E2150F0EC00F0DD
:10142000212A006E00C030F00BEC02F0150E215C9A
:10143000F4E1928480B448D01E6A1E501DEC00F086
:10144000000905E01E2A306E0BEC02F0F6D7010E03
:10145000316E326EF9EC01F01E6A1E5003EC01F0A1
:101460001E2A006E00C030F00BEC02F0100E1E5C65
:10147000F4E117C02DF016C02CF055DD02C011F0BC
:1014800001C010F01150260807E2FF0A03E11050D6
:101490000F0802E2116A106A11C01FF010C01EF09E
:1014A000216A206A270E236E0F0E226EB7DD02C05E
:1014B00011F001C010F017C01FF016C01EF011C0CF
:1014C00021F010C020F0B0DE31D1010E316E326E4D
:1014D000F9EC01F0060E1E6E2D0E306E0BEC02F0D4
:1014E0001E2EFAD71F6A1F5014EC01F01F2A006E3F
:1014F00000C030F00BEC02F0040E1F5CF4E1060EAD
:10150000206E2D0E306E0BEC02F0202EFAD7040E5A
:10151000216E215014EC01F0212A006E00C030F041
:101520000BEC02F0150E215CF4E1928480B448D0FB
:101530001E6A1E501DEC00F0000905E01E2A306EE8
:101540000BEC02F0F6D7010E316E326EF9EC01F0C1
:101550001E6A1E5027EC01F01E2A006E00C030F0FB
:101560000BEC02F0100E1E5CF4E119C02DF018C057
:101570002CF0D9DC02C00DF001C00CF00D500008B9
:1015800007E2FF0A03E10C50F40802E20D6A0C6A5C
:101590000DC01FF00CC01EF0216A206A010E236EE0
:1015A000F40E226E3BDD02C00DF001C00CF019C03C
:1015B0001FF018C01EF00DC021F00CC020F034DE6A
:1015C000B5D0010E316E326EF9EC01F0060E1E6ED2
:1015D0002D0E306E0BEC02F01E2EFAD71F6A1F5034
:1015E00038EC01F01F2A006E00C030F00BEC02F066
:1015F000040E1F5CF4E1060E206E2D0E306E0BEC17
:1016000002F0202EFAD7040E216E215038EC01F0A2
:10161000212A006E00C030F00BEC02F0150E215CA8
:10162000F4E1928480B448D01E6A1E501DEC00F094
:10163000000905E01E2A306E0BEC02F0F6D7010E11
:10164000316E326EF9EC01F01E6A1E504BEC01F067
:101650001E2A006E00C030F00BEC02F0100E1E5C73
:10166000F4E11BC02DF01AC02CF05DDC02C00FF0BD
:1016700001C00EF00F50000807E2FF0A03E10E5010
:10168000F40802E20F6A0E6A0FC01FF00EC01EF0CF
:10169000216A206A010E236EF40E226EBFDC02C0A6
:1016A0000FF001C00EF01BC01FF01AC01EF00FC0DB
:1016B00021F00EC020F0B8DD39D0010E316E326E4F
:1016C000F9EC01F0060E1E6E2D0E306E0BEC02F0E2
:1016D0001E2EFAD71F6A1F505CEC01F01F2A006E05
:1016E00000C030F00BEC02F0040E1F5CF4E1060EBB
:1016F000206E2D0E306E0BEC02F0202EFAD7040E69
:10170000216E21505CEC01F0212A006E00C030F007
:101710000BEC02F0110E215CF4E1040E226E200E9F
:10172000306E0BEC02F0222EFAD700D0FA0E316E9A
:101730007BEC01F0A8D51E6A1E501DEC00F00009DC
:1017400005E01E2A306E0BEC02F0F6D7A3EF0DF089
:10175000E8246B0FF66E170EF76ED8B0F72A0A0062
:10176000F550FA6E0800F550F96EDA125613D213DE
:10177000CA14C215BA16000E016EC250C70B011072
:10178000C26EC284C2B4FED7C3CF20F0C4CF21F052
:1017900020C001F021C002F0000C3A6A3B6A010E41
:1017A0003C6EDA6AD96A3F6A320E3E6EEA6A360EDB
:1017B000E96E3FC0E2FF3EC0E1FF3CC03DF0D89083
:1017C000E550EE02F3503A22F4503B223D2EF7D77B
:1017D0003AC0DEFF3BC03AF03B6AD8B03B2A3E2A13
:1017E000D8B43F2A3C2A3C500508E0E1000C006ACE
:1017F000016A026A036A366A376A386A396A35509A
:101800003410331032102CE0200E3A6ED8902E3661
:101810002F3630363136363637363836393635505B
:10182000395C08E13450385C05E13350375C02E143
:101830003250365C0FE33250365E3350D8A0333C22
:10184000375E3450D8A0343C385E3550D8A0353C93
:10185000395ED88000360136023603363A2ED6D7A6
:101860000000EA6A360EE96E000C2B6A2A6A23C071
:1018700029F022C028F017C02DF016C02CF093ECF0
:1018800007F001C000F002C001F0026A036A03C061
:101890002FF002C02EF001C02DF000C02CF0EACFD6
:1018A00031F0E9CF30F02BC035F02AC034F029C038
:1018B00033F028C032F003C039F002C038F001C064
:1018C00037F000C036F069DF31C0EAFF30C0E9FF11
:1018D00003C027F002C026F001C025F000C024F0AC
:1018E00027C031F026C030F025C02FF024C02EF0E4
:1018F000356A346A030E336EFF0E326E78DF03C032
:1019000027F002C026F001C025F000C024F024C05A
:1019100001F025C002F0000C17C02DF016C02CF00D
:1019200093EC07F002C026F001C025F02C6A2B6A68
:1019300020C02AF01FC029F025C000F026C001F009
:10194000026A036A03C030F002C02FF026C02EF0F6
:1019500025C02DF02CC035F02BC034F020C033F062
:101960001FC032F003C039F002C038F026C037F093
:1019700025C036F012DF03C02DF002C02CF001C0EC
:101980002BF000C02AF003C031F002C030F001C0DB
:101990002FF000C02EF0356A346A030E336EFF0E4E
:1019A000326E25DF03C024F002C023F001C022F014
:1019B00000C021F024C035F023C034F022C033F041
:1019C00021C032F0396A386A376A640E366EE5DE55
:1019D00003C02CF002C02BF001C02AF000C029F097
:1019E00003C031F002C030F001C02FF000C02EF073
:1019F000356A346A26C033F025C032F0F8DE00C004
:101A000001F0BDEF0DF0B7DE02C021F001C020F003
:101A100002C023F001C022F028DF02C01EF001C086
:101A20001DF019C02DF018C02CF093EC07F002C087
:101A30000DF001C00CF01BC02DF01AC02CF093EC7F
:101A400007F002C00FF001C00EF00E500C24016E22
:101A50000F500D20036E03501E5C06E303E101509E
:101A60001D5C02E31C801F801E500D5C05E303E13A
:101A70000C501D5C01E21C901F900D501E5C04E395
:101A800005E11D500C5C02E3000E01D0010E206E3A
:101A9000000E1CB0010E010802E0000E01D0010E84
:101AA0002014000A02E01F8001D01F90000E1FB01A
:101AB000010E01080FE1000E1CB2010E000A09E13F
:101AC00095968C96939A8A9A93988A8895948C8402
:101AD0001C820ED0000E1CB2010E010809E1959483
:101AE0008C9493988A98939A8A8A95968C861C925D
:101AF000FBEF0EF0F86AD09EEA6AE96AC180C18203
:101B0000C184C196810EAF6E260EAC6E900EAB6E88
:101B1000010E166E176A030E186E196A050E1A6EFC
:101B20001B6A5BEF03F09286000E80A6010E1D6E0D
:101B30009288000E80A8010E1D10000A06E0959202
:101B40008C8229EF09F095928C9215DE02C01EF06E
:101B500001C01DF002C023F001C022F086DE02C0E9
:101B600013F001C012F007DE02C01EF001C01DF02C
:101B700002C020F001C01FF0CFD6156A01C014F0DA
:101B80009488040E006E002EFED79486060E006E1A
:101B9000002EFED78B989498040E006E002EFED770
:101BA0008B969496D00E356E2DEC02F0030E356EAA
:101BB0002DEC02F09488040E006E002EFED7948661
:101BC000060E006E002EFED78B989498040E006EC1
:101BD000002EFED78B969496D10E356E2DEC02F02A
:101BE000010E006E64EC02F001507F0B1F6E1FC0EF
:101BF00024F097EC02F001C00BF0010E006E64ECD3
:101C000002F001503F0B1F6E1FC024F097EC02F052
:101C100001C008F0010E006E64EC02F001501F0BD1
:101C20001F6E1FC024F097EC02F001C009F0006A9B
:101C300064EC02F001C01EF001C024F097EC02F049
:101C400001C00AF094980000948682A6FED7040E84
:101C5000006E002EFED70000000000009488040EE5
:101C6000006E002EFED79488040E006E002EFED764
:101C70009486060E006E002EFED78B989498040E64
:101C8000006E002EFED78B969496D00E356E2DECFE
:101C900002F0356A2DEC02F09488040E006E002EDE
:101CA000FED79486060E006E002EFED78B98949871
:101CB000040E006E002EFED78B969496D10E356ED4
:101CC0002DEC02F0010E006E64EC02F001507F0B6F
:101CD0001F6E1FC024F097EC02F001C005F0010E4A
:101CE000006E64EC02F001507F0B1F6E1FC024F0E9
:101CF00097EC02F001C006F0006A64EC02F00150BB
:101D00003F0B1F6E1FC024F097EC02F001C007F0DC
:101D100094980000948682A6FED7040E006E002ED2
:101D2000FED70000000000009488040E006E002E14
:101D3000FED7010E316E326EF9EC01F0C80E316E35
:101D40007BEC01F008C01FF0010E206EF4EC03F0F4
:101D50002F0E306E0BEC02F009C01FF0010E206E4A
:101D6000F4EC03F0200E306E0BEC02F0200E306E1F
:101D70000BEC02F007C01FF0010E206EF4EC03F034
:101D80003A0E306E0BEC02F006C01FF0010E206E12
:101D9000F4EC03F03A0E306E0BEC02F005C01FF0CD
:101DA000010E206EF4EC03F00A0E306E0BEC02F024
:101DB000010EE96E13C028F012C027F0ADEC07F059
:101DC000040E1D6E1D500CEC00F01D2A006E00C0AC
:101DD00030F00BEC02F00B0E1D5CF4E1020EE96E2C
:101DE00015C028F014C027F0ADEC07F0250E306EBA
:0A1DF0000BEC02F008D697D60300B2
:020000040030CA
:0E00000000220F0E000101000FC00FE00F40A4
:00000001FF
